:020000020000FC
:1006E0000000C8C80000C4C4C2C2C0C0C1C1CBCBD6
:1006F0000000C9C9C7C7C5C5C3C30909E0E00000F8
:10070000000000000000E4E400007151312100000D
:10071000000000007A5A735361417757322200F08B
:10072000000063437858644465453424332300F162
:10073000000020207656664674547252352500F229
:1007400000006E4E624268486747795936260000BD
:10075000000000006D4D6A4A7555372738280000A3
:1007600000002C3C6B4B69496F4F30003929000069
:1007700000002E3E2F3F6C4C3B2B70502D3D000057
:1007800000005C5F3A2A000040605E7E00000000CE
:10079000E1D200000D0D5B7B00005D7D00000000DC
:1007A0000000000000000000E3E300000808E2E2AF
:1007B0000000B1A15C7CB4A4B7A700000000000059
:1007C000B0A02E7FB2A2B500B6A6B8A81B1BD1D18F
:1007D000CACA2B2BB3A32D2D2A2AB9A9D0D0000029
:1007E000000000000000C6C6ABAB00000000000027
:1007F00000000000000000000000000000000000F9
:100000000BC06CC108C007C006C005C004C085C1D4
:1000100002C001C000C018950FED0DBF0BE601BB7B
:10002000002702BB02E005BF08E90AB90CE009B9E4
:1000300033274BE074E588279927AA27BB27CC27CD
:1000400000E40BBF78942CC09B7FEE2496FD28C063
:1000500095FD1EC094FD20C090FD03C092FFF6CF19
:1000600003C093FD99F709C02E2D743521F0783522
:1000700011F01ED0E9CF35D0E7CFFC2C05D113D03D
:1000800091FF03C0FD2C00D10ED09E7F9D7FDCCF61
:100090009F7D082DE2D1D8CF9F7E082DEBD1D4CF04
:1000A0009F7B00D2D1CF9B7FEE2492FFFECF08959D
:1000B0005D9BFECF2CB908952F93229520632A33A0
:1000C00010F007E0200F5D9BFECF2CB92F912F7011
:1000D00020632A3310F007E0200F5D9BFECF2CB980
:1000E000089580FD8FC0203E11F48860BAC0213E83
:1000F00011F48061B6C0203F11F48160B2C0243198
:1001000071F483FD07C084FDACC0A0FDAAC0A1604E
:1001100020E94CC0A3FDA5C0A86023E947C0213158
:1001200061F483FD05C0A2FD9CC0A46022E93EC02D
:10013000A5FD97C0A06225E939C0223129F4A1FDAF
:1001400090C0A26021E932C0293529F4A4FD89C0FC
:10015000A06124E92BC0F3E0E0E7E20F2227F21FC1
:100160008894EE1FFF1F0A2F027111F483FF01C054
:10017000E160C895202D0A2F097051F0213440F01C
:100180002B3730F42B3518F0213608F4F2CF2F71CD
:10019000203B60F02A3B50F4B1FF03C02F70206376
:1001A00005C02F70206A253A09F420E02F3319F496
:1001B00083FD2FE218C0213D19F484FD2AEA06C010
:1001C000203D21F40A2F097009F02AEAB2FF0BC082
:1001D000213420F02B3510F4206205C0213618F0B0
:1001E0002B3708F42F7D203051F0783511F020386E
:1001F00008F45EDF203D18F0233D08F433D0877FFC
:100200008F7E2FC084FF03C0273759F526C02431C5
:1002100051F483FD05C084FD24C0AE7F26E918C0DB
:10022000A77F29E915C0213141F483FD03C0AB7FCD
:1002300028E90EC0AF7D2BE90BC0223119F4AD7F48
:1002400027E906C0293519F4AF7E2AE901C005C0A7
:10025000783511F0203808F42BDF8E7F877F8F7E72
:1002600000C00895203D11F401E007C0213D11F4C4
:1002700002E003C0223D39F404E0B02791609260AF
:100280000DEEC02EDB2E0895F894929894988A9AD9
:1002900000E800000A95E9F78C9A8A9868E05527EB
:1002A000C5D0F79410F08C9A02C08C985395BED0AC
:1002B0006A95B9F750FD02C08C9801C08C9AB6D0EF
:1002C0008C98B4D0849B03C00FEFF02EDDCF829BBF
:1002D000FECF33274BE08827789408950FB60F920E
:1002E0001F93986082FD0BC04B3028F4433018F008
:1002F00036958499306813E015BF84600AC012E017
:1003000015BF8B7F4A9529F4E32E33274BE0946089
:10031000977F1F910F900FBE18950FB60F921F93E6
:100320000F931CB1CC2309F054C0163559F420E5C5
:10033000BFDE20E5BDDE23E4BBDE21E4B9DE2BE237
:10034000B7DE6FC01D3429F473E504EF9160C02E51
:1003500068C0133511F473E564C0143511F474E505
:1003600060C0183511F478E55CC01C3421F42B2FE3
:1003700020639EDE56C01B3461F42A2F2770206351
:1003800097DE2A2F2695269526952770206390DEE6
:1003900048C0123531F491600FEFC02EAA27BB2759
:1003A00040C0153411F4C8603CC0113311F4C16071
:1003B00038C0123311F4C26034C0103511F4C0617A
:1003C00030C0113511F4C0622CC0153551F5906460
:1003D00028C0C3FF08C0916092600DEEC02E177058
:1003E000D12ECC271EC0C0FF04C09160C12ECC27E7
:1003F00018C0C2FF05C091609260D12ECC2711C0F9
:10040000C1FF03C0C12EC4600CC0C4FF04C0812E54
:100410009061CC2706C0C5FF03C0812E9062CC2717
:1004200000C00F911F910F900FBE1895829BFECFB9
:100430008299FECF0895AA24A7BA9398959A969A7E
:100440000000A6B296980A2D089500E4B02EF3DFBE
:10045000007811F0BA94D9F70895902EF6DF9398AA
:10046000959898BAAA24A094A7BA98BA969A000028
:1004700096980895902EE9DF939A959898BAAA24B1
:10048000A094A7BA98BA969A000096980895DDDFCE
:10049000AA24A7BA939A959A969A000006B3902E2A
:1004A000969808951FD01ED000E3902ED8DF1DD05F
:1004B00000E3902ED4DF1FD000E3902ED0DF1BD0BE
:1004C00008E3902ECCDF08E0C8DF0FD001E0C5DFE5
:1004D00006E0C3DF02E0C1DF0CE0BFDF06D00CE0C6
:1004E000BCDF08950AEFB02E0BC006E9B02E08C09D
:1004F00002E3B02E05C00AE0B02E02C001E0B02E2B
:1005000008EC00000A95E9F7BA94D1F70895BB24E6
:10051000B0948894B7948894B794BA94F1F70895F6
:00000001FF
